:020000020000FC
:100000000C9434000C9434000C9434000C94F200E2
:100010000C9434000C9434000C9434000C94340090
:100020000C9434000C9434000C9434000C945F0154
:100030000C9434000C9434000C94FC000C943400A8
:100040000C9434000C9434000C9434000C94340060
:100050000C9434000C9462010C9434000C94340021
:100060000C9434000C943400F89404E00EBF0FEFAD
:100070000DBF009160000861009360000FE00093E5
:1000800060000AE01DE004B915B90FE310E007B9FC
:1000900018B900E010E80AB91BB92224B1E0A0E0C9
:1000A0002D92AF3FE9F7BED103D202E804BD04E0D0
:1000B00005BD0DE707BD02E8009380000CE9009341
:1000C000810017E00FEF10938700009386002092C5
:1000D00089002092880002E000936E0002E0009305
:1000E0006F0001E00093680001E000936B000DECED
:1000F00000937A0006EC00937C00F6E0E0E900272C
:100100000064F7D12FD20591003219F00CD22AD217
:10011000FACF8824662701E0009323010CE20093C4
:100120002401622C05E0702E12E000E010932501FE
:1001300000932601789403E50093000105E60093FF
:10014000010104E7009302010AE30093030103E4C1
:100150000093100105E70093110102E700931201DB
:100160000AE300931301A895AAD124D1E1D0BBD012
:1001700010912301009124011DD2E0920501D0923B
:100180000601C0920701109121010091220112D2B3
:1001900010912101123020F00DE2E02ED02EC02E61
:1001A000E0921501D0921601C0921701122D072D71
:1001B00001D2D0920B01C0920C010AE300930D0111
:1001C000122D062DF7D1D0920E01C0920F012B9A5D
:1001D000772039F4662011F42B98C5CF082D00FF45
:1001E0002B98C1CF1A9B1895189903C0F49AF598CB
:1001F0001895F59AF4981895BFB6BF920F931F9370
:100200002F933F93F29B0BC04395453041F4F298F6
:1002100000917A00006400937A00442701C0F09AAC
:100220009A94C9F50AEF902E8394F69934C0009100
:1002300028011091270120912601309125010A50B3
:1002400012092017310738F095E1090F121D201708
:10025000310708F403C0622C05E0702E30932701AB
:10026000209328016A940FEF6016A9F40BE3602E27
:100270007A940FEF701679F400912301009329010D
:100280000091240100932A0120922301209224014D
:10029000722C622CF69A0FEFA01609F0A3944F9BD4
:1002A00003C0AA24F19804C008E2A01609F4F19A48
:1002B0003F912F911F910F91BF90BFBE1895F29A59
:1002C000F39A1895BFB6BF920F931F9300917800D1
:1002D0001091790000932201109321011F910F9139
:1002E000BF90BFBE189510912501009126012227CD
:1002F0000332120520F0035212092395F9CFF5E0DD
:10030000E4EF293108F029E106E0209FE00DF11D1E
:10031000059100931B01059100931C010591009329
:100320001D01059100931E01059100931F01089581
:10033000F49B13C0F69911C0622C05E0702EF4985E
:10034000F0912301E091240101E0EE35F00728F45B
:100350003A96F0932301E0932401F59B13C0F6999C
:1003600011C0622C05E0702EF598F0912301E09108
:10037000240100E0E03FF00729F03A97F0932301D1
:10038000E0932401F19B15C0F198622C05E0702EDA
:10039000F69B0895F698009129010093230100919E
:1003A0002A010093240112E000E01093250100933C
:1003B00026010895F39B0895F3981091210100916F
:1003C0002201209123013091240103171207A8F084
:1003D00041F1009126011091250120E030E0021743
:1003E0001307F9F001501209109389000093880057
:1003F0001093250100932601089500912601109184
:10040000250120E733E00217130758F421E0020F1B
:10041000121D10938900009388001093250100930A
:1004200026010895AAD0A9D000E3029508B90000DA
:1004300000000000459A000000000000459892D09E
:10044000A8959BD000E3029508B9000000000000C9
:10045000459A00000000000045988FD0A89500E361
:10046000029508B9000000000000459A0000000055
:100470000000459877D000E2029508B9000000001E
:100480000000459A00000000000045986BD008E28B
:1004900030D068D00CE02DD065D0A89501E029D0EF
:1004A0006CD06BD06AD006E0662723D066D0089562
:1004B000B1E0A0E000E20D93A032E9F70895F09BCF
:1004C0000895F098D1E0C0E0C60FD21D603021F44D
:1004D00000E000680ED046D0603121F400E40068EE
:1004E00008D040D008811FD06395603208F066279D
:1004F0000895102F12951F7018B900000000000019
:10050000459A0000000000004598102F1F7018B990
:10051000000000000000459A00000000000045981F
:10052000112718B90895102F12951F70449A106161
:1005300018B9000000000000459A0000000000000B
:1005400000004598102F1F70106118B900000000BE
:100550000000459A000000000000000045981127A7
:1005600018B9089502E80A95F1F7089500271EE1E9
:100570000A95F1F71A95E1F70895002711270A95D2
:10058000F1F71A95E1F70895102F107F1295D12EEB
:1005900010E3D10E1AE3D11610F017E0D10E102F90
:1005A0001F70C12E10E3C10E1AE3C11610F017E040
:1005B000C10E0895CC24DD24EE24FF24083E23E060
:1005C000120720F0085E1340F394F8CF043620E0C1
:1005D000120720F004561040E394F8CF0A3018F0C8
:1005E0000A50D394FBCFC02E00E3F00EE00ED00EE5
:1005F000C00E08950000000000000100000000008F
:1006000002000000000003000000000004000000E1
:1006100000000500000000000501000000000502C8
:1006200000000000050300000000050400000000B9
:100630000505000000000505010000000505020099
:100640000000050503000000050504000000050585
:100650000500000005050501000005050502000074
:100660000505050300000505050400000505050551
:100670000000050505050100050505050200050545
:10068000050503000505050504000505050505002C
:1006900000000015000000001010101510101000D0
:1006A0001818181D181818001C1C1C1D1C1C1C00D8
:1006B0001E1E1E1F1E1E1E001F1F1F1F1F1F1F008E
:0206C000200018
:00000001FF
